 j2pkcs11

 Timestamp is df4488e9 (reproducible build file hash)

 Preferred load address is 10000000

 Start         Length     Name                   Class
 0001:00000000 00008ee9H .text$mn                CODE
 0002:00000000 000000c4H .idata$5                DATA
 0002:000000c4 00000008H .00cfg                  DATA
 0002:000000cc 00000004H .CRT$XCA                DATA
 0002:000000d0 00000004H .CRT$XCZ                DATA
 0002:000000d4 00000004H .CRT$XIA                DATA
 0002:000000d8 00000004H .CRT$XIZ                DATA
 0002:000000dc 00000004H .CRT$XPA                DATA
 0002:000000e0 00000004H .CRT$XPZ                DATA
 0002:000000e4 00000004H .CRT$XTA                DATA
 0002:000000e8 00000008H .CRT$XTZ                DATA
 0002:000000ec 00000000H .gfids$y                DATA
 0002:000000f0 00001310H .rdata                  DATA
 0002:00001400 00000000H .rdata$CastGuardVftablesA DATA
 0002:00001400 00000000H .rdata$CastGuardVftablesC DATA
 0002:00001400 00000004H .rdata$sxdata           DATA
 0002:00001404 00000064H .rdata$voltmd           DATA
 0002:00001468 000002a0H .rdata$zzzdbg           DATA
 0002:00001708 00000004H .rtc$IAA                DATA
 0002:0000170c 00000004H .rtc$IZZ                DATA
 0002:00001710 00000004H .rtc$TAA                DATA
 0002:00001714 00000004H .rtc$TZZ                DATA
 0002:00001718 00000088H .xdata$x                DATA
 0002:000017a0 000012ecH .edata                  DATA
 0002:00002a8c 00000078H .idata$2                DATA
 0002:00002b04 00000014H .idata$3                DATA
 0002:00002b18 000000c4H .idata$4                DATA
 0002:00002bdc 000003ccH .idata$6                DATA
 0003:00000000 00000308H .data                   DATA
 0003:00000308 000003a4H .bss                    DATA
 0004:00000000 00000060H .rsrc$01                DATA
 0004:00000060 00000330H .rsrc$02                DATA

  Address         Publics by Value              Rva+Base       Lib:Object

 0000:00000000       ___AbsoluteZero            00000000     <absolute>
 0000:00000000       ___arm64x_extra_rfe_table  00000000     <absolute>
 0000:00000000       ___arm64x_extra_rfe_table_size 00000000     <absolute>
 0000:00000000       ___arm64x_native_entrypoint 00000000     <absolute>
 0000:00000000       ___arm64x_redirection_metadata 00000000     <absolute>
 0000:00000000       ___arm64x_redirection_metadata_count 00000000     <absolute>
 0000:00000000       ___dynamic_value_reloc_table 00000000     <absolute>
 0000:00000000       ___enclave_config          00000000     <absolute>
 0000:00000000       ___guard_check_icall_a64n_fptr 00000000     <absolute>
 0000:00000000       ___guard_eh_cont_count     00000000     <absolute>
 0000:00000000       ___guard_eh_cont_table     00000000     <absolute>
 0000:00000000       ___guard_fids_count        00000000     <absolute>
 0000:00000000       ___guard_fids_table        00000000     <absolute>
 0000:00000000       ___guard_iat_count         00000000     <absolute>
 0000:00000000       ___guard_iat_table         00000000     <absolute>
 0000:00000000       ___guard_longjmp_count     00000000     <absolute>
 0000:00000000       ___guard_longjmp_table     00000000     <absolute>
 0000:00000000       ___hybrid_auxiliary_delayload_iat 00000000     <absolute>
 0000:00000000       ___hybrid_auxiliary_delayload_iat_copy 00000000     <absolute>
 0000:00000000       ___hybrid_auxiliary_iat    00000000     <absolute>
 0000:00000000       ___hybrid_auxiliary_iat_copy 00000000     <absolute>
 0000:00000000       ___hybrid_code_map         00000000     <absolute>
 0000:00000000       ___hybrid_code_map_count   00000000     <absolute>
 0000:00000000       ___hybrid_image_info_bitfield 00000000     <absolute>
 0000:00000000       ___x64_code_ranges_to_entry_points 00000000     <absolute>
 0000:00000000       ___x64_code_ranges_to_entry_points_count 00000000     <absolute>
 0000:00000001       ___safe_se_handler_count   00000001     <absolute>
 0000:00000100       ___guard_flags             00000100     <absolute>
 0000:00000000       ___ImageBase               10000000     <linker-defined>
 0001:00000000       _Java_sun_security_pkcs11_Secmod_nssGetModuleList@20 10001000 f   j2secmod.obj
 0001:000001a0       _Java_sun_security_pkcs11_Secmod_nssInitialize@28 100011a0 f   j2secmod.obj
 0001:000002da       _Java_sun_security_pkcs11_Secmod_nssVersionCheck@20 100012da f   j2secmod.obj
 0001:00000334       _Java_sun_security_pkcs11_Secmod_nssGetLibraryHandle@12 10001334 f   j2secmod_md.obj
 0001:0000036c       _Java_sun_security_pkcs11_Secmod_nssLoadLibrary@12 1000136c f   j2secmod_md.obj
 0001:000003e2       ___local_stdio_printf_options 100013e2 f i j2secmod_md.obj
 0001:000003e8       __snprintf                 100013e8 f i j2secmod_md.obj
 0001:00000402       __vsnprintf                10001402 f i j2secmod_md.obj
 0001:0000041d       __vsnprintf_l              1000141d f i j2secmod_md.obj
 0001:00000450       _findFunction              10001450 f   j2secmod_md.obj
 0001:000004b1       _ckAttributePtrToJAttribute 100014b1 f   p11_convert.obj
 0001:00000537       _ckAttributeValueToJObject 10001537 f   p11_convert.obj
 0001:00000741       _ckDatePtrToJDateObject    10001741 f   p11_convert.obj
 0001:0000080f       _ckSessionInfoPtrToJSessionInfo 1000180f f   p11_convert.obj
 0001:00000878       _ckVersionPtrToJVersion    10001878 f   p11_convert.obj
 0001:000008d7       _copyBackPBEInitializationVector 100018d7 f   p11_convert.obj
 0001:000009ed       _jAesCtrParamsToCKAesCtrParamPtr 100019ed f   p11_convert.obj
 0001:00000b1a       _jAttributeToCKAttribute   10001b1a f   p11_convert.obj
 0001:00000bb3       _jCCMParamsToCKCCMParamPtr 10001bb3 f   p11_convert.obj
 0001:00000d3d       _jDateObjectToCKDatePtr    10001d3d f   p11_convert.obj
 0001:00000f89       _jEcdh1DeriveParamToCKEcdh1DeriveParamPtr 10001f89 f   p11_convert.obj
 0001:000010cc       _jEcdh2DeriveParamToCKEcdh2DeriveParamPtr 100020cc f   p11_convert.obj
 0001:000012b6       _jGCMParamsToCKGCMParamPtr 100022b6 f   p11_convert.obj
 0001:00001414       _jMechParamToCKMechParamPtr 10002414 f   p11_convert.obj
 0001:00001495       _jMechParamToCKMechParamPtrSlow 10002495 f   p11_convert.obj
 0001:000017b6       _jMechanismToCKMechanismPtr 100027b6 f   p11_convert.obj
 0001:00001830       _jPbeParamToCKPbeParamPtr  10002830 f   p11_convert.obj
 0001:000019c2       _jPkcs5Pbkd2ParamToCKPkcs5Pbkd2ParamPtr 100029c2 f   p11_convert.obj
 0001:00001b6b       _jRsaPkcsOaepParamToCKRsaPkcsOaepParamPtr 10002b6b f   p11_convert.obj
 0001:00001ca7       _jRsaPkcsPssParamToCKRsaPkcsPssParamPtr 10002ca7 f   p11_convert.obj
 0001:00001d82       _jSalsaChaChaPolyParamsToCKSalsaChaChaPolyParamPtr 10002d82 f   p11_convert.obj
 0001:00001e9f       _jSsl3KeyMatParamToCKSsl3KeyMatParamPtr 10002e9f f   p11_convert.obj
 0001:00001f30       _jSsl3MasterKeyDeriveParamToCKSsl3MasterKeyDeriveParamPtr 10002f30 f   p11_convert.obj
 0001:00001faf       _jTls12KeyMatParamToCKTls12KeyMatParamPtr 10002faf f   p11_convert.obj
 0001:00002071       _jTls12MasterKeyDeriveParamToCKTls12MasterKeyDeriveParamPtr 10003071 f   p11_convert.obj
 0001:00002123       _jTlsMacParamsToCKTlsMacParamPtr 10003123 f   p11_convert.obj
 0001:000021fe       _jTlsPrfParamsToCKTlsPrfParamPtr 100031fe f   p11_convert.obj
 0001:00002370       _jVersionToCKVersionPtr    10003370 f   p11_convert.obj
 0001:00002401       _jX942Dh1DeriveParamToCKX942Dh1DeriveParamPtr 10003401 f   p11_convert.obj
 0001:00002544       _jX942Dh2DeriveParamToCKX942Dh2DeriveParamPtr 10003544 f   p11_convert.obj
 0001:00002742       _keyMatParamToCKKeyMatParam 10003742 f   p11_convert.obj
 0001:00002a4d       _masterKeyDeriveParamToCKMasterKeyDeriveParam 10003a4d f   p11_convert.obj
 0001:00002bb0       _Java_sun_security_pkcs11_wrapper_PKCS11_C_1Decrypt@56 10003bb0 f   p11_crypt.obj
 0001:00002cbd       _Java_sun_security_pkcs11_wrapper_PKCS11_C_1DecryptFinal@36 10003cbd f   p11_crypt.obj
 0001:00002d4c       _Java_sun_security_pkcs11_wrapper_PKCS11_C_1DecryptInit@28 10003d4c f   p11_crypt.obj
 0001:00002da6       _Java_sun_security_pkcs11_wrapper_PKCS11_C_1DecryptUpdate@56 10003da6 f   p11_crypt.obj
 0001:00002eb3       _Java_sun_security_pkcs11_wrapper_PKCS11_C_1Encrypt@56 10003eb3 f   p11_crypt.obj
 0001:00002fbd       _Java_sun_security_pkcs11_wrapper_PKCS11_C_1EncryptFinal@36 10003fbd f   p11_crypt.obj
 0001:0000304c       _Java_sun_security_pkcs11_wrapper_PKCS11_C_1EncryptInit@28 1000404c f   p11_crypt.obj
 0001:000030a3       _Java_sun_security_pkcs11_wrapper_PKCS11_C_1EncryptUpdate@56 100040a3 f   p11_crypt.obj
 0001:000031ad       _Java_sun_security_pkcs11_wrapper_PKCS11_C_1GCMDecryptInitWithRetry@32 100041ad f   p11_crypt.obj
 0001:00003260       _Java_sun_security_pkcs11_wrapper_PKCS11_C_1GCMEncryptInitWithRetry@32 10004260 f   p11_crypt.obj
 0001:0000330d       _Java_sun_security_pkcs11_wrapper_PKCS11_C_1DigestFinal@28 1000430d f   p11_digest.obj
 0001:00003389       _Java_sun_security_pkcs11_wrapper_PKCS11_C_1DigestInit@20 10004389 f   p11_digest.obj
 0001:000033e0       _Java_sun_security_pkcs11_wrapper_PKCS11_C_1DigestKey@24 100043e0 f   p11_digest.obj
 0001:00003410       _Java_sun_security_pkcs11_wrapper_PKCS11_C_1DigestSingle@44 10004410 f   p11_digest.obj
 0001:00003599       _Java_sun_security_pkcs11_wrapper_PKCS11_C_1DigestUpdate@36 10004599 f   p11_digest.obj
 0001:000036ed       _Java_sun_security_pkcs11_wrapper_PKCS11_C_1GenerateRandom@20 100046ed f   p11_digest.obj
 0001:0000375c       _Java_sun_security_pkcs11_wrapper_PKCS11_C_1SeedRandom@20 1000475c f   p11_digest.obj
 0001:000037c5       _JNI_OnLoad@8              100047c5 f   p11_general.obj
 0001:000037d6       _Java_sun_security_pkcs11_wrapper_PKCS11_C_1Finalize@12 100047d6 f   p11_general.obj
 0001:00003800       _Java_sun_security_pkcs11_wrapper_PKCS11_C_1GetInfo@8 10004800 f   p11_general.obj
 0001:0000386b       _Java_sun_security_pkcs11_wrapper_PKCS11_C_1GetMechanismInfo@24 1000486b f   p11_general.obj
 0001:000038cd       _Java_sun_security_pkcs11_wrapper_PKCS11_C_1GetMechanismList@16 100048cd f   p11_general.obj
 0001:00003962       _Java_sun_security_pkcs11_wrapper_PKCS11_C_1GetSlotInfo@16 10004962 f   p11_general.obj
 0001:000039c1       _Java_sun_security_pkcs11_wrapper_PKCS11_C_1GetSlotList@12 100049c1 f   p11_general.obj
 0001:00003a60       _Java_sun_security_pkcs11_wrapper_PKCS11_C_1GetTokenInfo@16 10004a60 f   p11_general.obj
 0001:00003ac8       _Java_sun_security_pkcs11_wrapper_PKCS11_C_1Initialize@12 10004ac8 f   p11_general.obj
 0001:00003b18       _Java_sun_security_pkcs11_wrapper_PKCS11_finalizeLibrary@8 10004b18 f   p11_general.obj
 0001:00003b1b       _Java_sun_security_pkcs11_wrapper_PKCS11_freeMechanism@16 10004b1b f   p11_general.obj
 0001:00003b36       _Java_sun_security_pkcs11_wrapper_PKCS11_initializeLibrary@12 10004b36 f   p11_general.obj
 0001:00003b69       _ckInfoPtrToJInfo          10004b69 f   p11_general.obj
 0001:00003c6d       _ckMechanismInfoPtrToJMechanismInfo 10004c6d f   p11_general.obj
 0001:00003cd2       _ckSlotInfoPtrToJSlotInfo  10004cd2 f   p11_general.obj
 0001:00003dd6       _ckTokenInfoPtrToJTokenInfo 10004dd6 f   p11_general.obj
 0001:000040ac       _fetchClass                100050ac f   p11_general.obj
 0001:000040cc       _prefetchFields            100050cc f   p11_general.obj
 0001:00004184       _Java_sun_security_pkcs11_wrapper_PKCS11_C_1DeriveKey@32 10005184 f   p11_keymgmt.obj
 0001:000042ff       _Java_sun_security_pkcs11_wrapper_PKCS11_C_1GenerateKey@24 100052ff f   p11_keymgmt.obj
 0001:00004408       _Java_sun_security_pkcs11_wrapper_PKCS11_C_1GenerateKeyPair@28 10005408 f   p11_keymgmt.obj
 0001:00004574       _Java_sun_security_pkcs11_wrapper_PKCS11_C_1UnwrapKey@36 10005574 f   p11_keymgmt.obj
 0001:0000468b       _Java_sun_security_pkcs11_wrapper_PKCS11_C_1WrapKey@36 1000568b f   p11_keymgmt.obj
 0001:000047d2       _Java_sun_security_pkcs11_wrapper_PKCS11_createNativeKey@32 100057d2 f   p11_keymgmt.obj
 0001:00004953       _Java_sun_security_pkcs11_wrapper_PKCS11_getNativeKeyInfo@36 10005953 f   p11_keymgmt.obj
 0001:000051a3       _copyBackTLSPrfParams      100061a3 f   p11_keymgmt.obj
 0001:000052ab       _ssl3CopyBackClientVersion 100062ab f   p11_keymgmt.obj
 0001:000052d0       _ssl3CopyBackKeyMatParams  100062d0 f   p11_keymgmt.obj
 0001:000052f9       _tls12CopyBackClientVersion 100062f9 f   p11_keymgmt.obj
 0001:0000531e       _tls12CopyBackKeyMatParams 1000631e f   p11_keymgmt.obj
 0001:00005347       _Java_sun_security_pkcs11_wrapper_PKCS11_connect@16 10006347 f   p11_md.obj
 0001:000054cc       _Java_sun_security_pkcs11_wrapper_PKCS11_disconnect@8 100064cc f   p11_md.obj
 0001:000054f6       _callJCreateMutex          100064f6 f   p11_mutex.obj
 0001:0000565f       _callJDestroyMutex         1000665f f   p11_mutex.obj
 0001:000057c9       _callJLockMutex            100067c9 f   p11_mutex.obj
 0001:00005925       _callJUnlockMutex          10006925 f   p11_mutex.obj
 0001:00005a81       _makeCKInitArgsAdapter     10006a81 f   p11_mutex.obj
 0001:00005c5f       _Java_sun_security_pkcs11_wrapper_PKCS11_C_1CopyObject@28 10006c5f f   p11_objmgmt.obj
 0001:00005cdf       _Java_sun_security_pkcs11_wrapper_PKCS11_C_1CreateObject@20 10006cdf f   p11_objmgmt.obj
 0001:00005d5c       _Java_sun_security_pkcs11_wrapper_PKCS11_C_1DestroyObject@24 10006d5c f   p11_objmgmt.obj
 0001:00005d89       _Java_sun_security_pkcs11_wrapper_PKCS11_C_1FindObjects@24 10006d89 f   p11_objmgmt.obj
 0001:00005e0c       _Java_sun_security_pkcs11_wrapper_PKCS11_C_1FindObjectsFinal@16 10006e0c f   p11_objmgmt.obj
 0001:00005e36       _Java_sun_security_pkcs11_wrapper_PKCS11_C_1FindObjectsInit@20 10006e36 f   p11_objmgmt.obj
 0001:00005e9e       _Java_sun_security_pkcs11_wrapper_PKCS11_C_1GetAttributeValue@28 10006e9e f   p11_objmgmt.obj
 0001:000060d4       _Java_sun_security_pkcs11_wrapper_PKCS11_C_1SetAttributeValue@28 100070d4 f   p11_objmgmt.obj
 0001:0000613f       _snprintf                  1000713f f i p11_objmgmt.obj
 0001:00006159       _vsnprintf                 10007159 f i p11_objmgmt.obj
 0001:0000618b       _Java_sun_security_pkcs11_wrapper_PKCS11_C_1CloseSession@16 1000718b f   p11_sessmgmt.obj
 0001:000061ec       _Java_sun_security_pkcs11_wrapper_PKCS11_C_1GetOperationState@16 100071ec f   p11_sessmgmt.obj
 0001:0000627d       _Java_sun_security_pkcs11_wrapper_PKCS11_C_1GetSessionInfo@16 1000727d f   p11_sessmgmt.obj
 0001:000062dc       _Java_sun_security_pkcs11_wrapper_PKCS11_C_1Login@28 100072dc f   p11_sessmgmt.obj
 0001:00006345       _Java_sun_security_pkcs11_wrapper_PKCS11_C_1Logout@16 10007345 f   p11_sessmgmt.obj
 0001:0000636f       _Java_sun_security_pkcs11_wrapper_PKCS11_C_1OpenSession@32 1000736f f   p11_sessmgmt.obj
 0001:0000643a       _Java_sun_security_pkcs11_wrapper_PKCS11_C_1SetOperationState@36 1000743a f   p11_sessmgmt.obj
 0001:000064a6       _notifyCallback            100074a6 f   p11_sessmgmt.obj
 0001:000065bb       _putNotifyEntry            100075bb f   p11_sessmgmt.obj
 0001:00006631       _removeNotifyEntry         10007631 f   p11_sessmgmt.obj
 0001:000066a1       _Java_sun_security_pkcs11_wrapper_PKCS11_C_1Sign@20 100076a1 f   p11_sign.obj
 0001:000067d4       _Java_sun_security_pkcs11_wrapper_PKCS11_C_1SignFinal@20 100077d4 f   p11_sign.obj
 0001:000068d4       _Java_sun_security_pkcs11_wrapper_PKCS11_C_1SignInit@28 100078d4 f   p11_sign.obj
 0001:0000694f       _Java_sun_security_pkcs11_wrapper_PKCS11_C_1SignRecover@40 1000794f f   p11_sign.obj
 0001:00006ae0       _Java_sun_security_pkcs11_wrapper_PKCS11_C_1SignRecoverInit@28 10007ae0 f   p11_sign.obj
 0001:00006b5b       _Java_sun_security_pkcs11_wrapper_PKCS11_C_1SignUpdate@36 10007b5b f   p11_sign.obj
 0001:00006caf       _Java_sun_security_pkcs11_wrapper_PKCS11_C_1Verify@24 10007caf f   p11_sign.obj
 0001:00006d50       _Java_sun_security_pkcs11_wrapper_PKCS11_C_1VerifyFinal@20 10007d50 f   p11_sign.obj
 0001:00006db9       _Java_sun_security_pkcs11_wrapper_PKCS11_C_1VerifyInit@28 10007db9 f   p11_sign.obj
 0001:00006e34       _Java_sun_security_pkcs11_wrapper_PKCS11_C_1VerifyRecover@40 10007e34 f   p11_sign.obj
 0001:00006fc5       _Java_sun_security_pkcs11_wrapper_PKCS11_C_1VerifyRecoverInit@28 10007fc5 f   p11_sign.obj
 0001:00007040       _Java_sun_security_pkcs11_wrapper_PKCS11_C_1VerifyUpdate@36 10008040 f   p11_sign.obj
 0001:00007195       __vfprintf_l               10008195 f i p11_util.obj
 0001:000071b9       _ckAssertReturnValueOK     100081b9 f   p11_util.obj
 0001:000071cc       _ckAssertReturnValueOK2    100081cc f   p11_util.obj
 0001:00007265       _ckBBoolPtrToJBooleanObject 10008265 f   p11_util.obj
 0001:000072b5       _ckByteArrayToJByteArray   100082b5 f   p11_util.obj
 0001:000072e7       _ckCharArrayToJCharArray   100082e7 f   p11_util.obj
 0001:000072e7       _ckUTF8CharArrayToJCharArray 100082e7 f   p11_util.obj
 0001:00007358       _ckULongArrayToJLongArray  10008358 f   p11_util.obj
 0001:000073cc       _ckULongPtrToJLongObject   100083cc f   p11_util.obj
 0001:00007415       _createLockObject          10008415 f   p11_util.obj
 0001:00007461       _fprintf                   10008461 f i p11_util.obj
 0001:00007479       _freeCKAttributeArray      10008479 f   p11_util.obj
 0001:000074b1       _freeCKMechanismPtr        100084b1 f   p11_util.obj
 0001:000075cd       _getFunctionList           100085cd f   p11_util.obj
 0001:000075f7       _getModuleEntry            100085f7 f   p11_util.obj
 0001:00007619       _jAttributeArrayToCKAttributeArray 10008619 f   p11_util.obj
 0001:00007735       _jBooleanArrayToCKBBoolArray 10008735 f   p11_util.obj
 0001:000077f2       _jBooleanObjectToCKBBoolPtr 100087f2 f   p11_util.obj
 0001:0000785a       _jByteArrayToCKByteArray   1000885a f   p11_util.obj
 0001:000078da       _jByteObjectToCKBytePtr    100088da f   p11_util.obj
 0001:00007938       _jCharArrayToCKCharArray   10008938 f   p11_util.obj
 0001:00007938       _jCharArrayToCKUTF8CharArray 10008938 f   p11_util.obj
 0001:000079f1       _jCharObjectToCKCharPtr    100089f1 f   p11_util.obj
 0001:00007a50       _jIntegerObjectToCKULongPtr 10008a50 f   p11_util.obj
 0001:00007aae       _jLongArrayToCKULongArray  10008aae f   p11_util.obj
 0001:00007b67       _jLongObjectToCKULongPtr   10008b67 f   p11_util.obj
 0001:00007bc9       _jObjectToPrimitiveCKObjectPtr 10008bc9 f   p11_util.obj
 0001:00007f5b       _jStringToCKUTF8CharArray  10008f5b f   p11_util.obj
 0001:00007fdb       _printDebug                10008fdb f   p11_util.obj
 0001:00008023       _putModuleEntry            10009023 f   p11_util.obj
 0001:0000804f       _removeModuleEntry         1000904f f   p11_util.obj
 0001:00008083       _throwByName               10009083 f   p11_util.obj
 0001:000080a3       _throwIOException          100090a3 f   p11_util.obj
 0001:000080b9       _throwNullPointerException 100090b9 f   p11_util.obj
 0001:000080cf       _throwOutOfMemoryError     100090cf f   p11_util.obj
 0001:000080e5       _throwPKCS11RuntimeException 100090e5 f   p11_util.obj
 0001:000080fb       _updateGCMParams           100090fb f   p11_util.obj
 0001:00008194       @__security_check_cookie@4 10009194 f   MSVCRT:secchk.obj
 0001:000081b0       __alloca_probe             100091b0 f   MSVCRT:chkstk.obj
 0001:000081b0       __chkstk                   100091b0 f   MSVCRT:chkstk.obj
 0001:0000851b       __DllMainCRTStartup@12     1000951b f   MSVCRT:dll_dllmain.obj
 0001:0000853e       ___raise_securityfailure   1000953e f   MSVCRT:gs_report.obj
 0001:00008566       ___report_gsfailure        10009566 f   MSVCRT:gs_report.obj
 0001:000086ad       ___security_init_cookie    100096ad f   MSVCRT:gs_support.obj
 0001:000086f8       _DllMain@12                100096f8 f   MSVCRT:dll_dllmain_stub.obj
 0001:0000871a       ?__scrt_initialize_type_info@@YAXXZ 1000971a f   MSVCRT:tncleanup.obj
 0001:00008726       ?__scrt_uninitialize_type_info@@YAXXZ 10009726 f   MSVCRT:tncleanup.obj
 0001:00008732       ___local_stdio_scanf_options 10009732 f i MSVCRT:default_local_stdio_options.obj
 0001:00008738       ___scrt_initialize_default_local_stdio_options 10009738 f   MSVCRT:default_local_stdio_options.obj
 0001:00008799       ___scrt_acquire_startup_lock 10009799 f   MSVCRT:utility.obj
 0001:000087cb       ___scrt_dllmain_after_initialize_c 100097cb f   MSVCRT:utility.obj
 0001:000087f6       ___scrt_dllmain_before_initialize_c 100097f6 f   MSVCRT:utility.obj
 0001:00008804       ___scrt_dllmain_crt_thread_attach 10009804 f   MSVCRT:utility.obj
 0001:00008823       ___scrt_dllmain_crt_thread_detach 10009823 f   MSVCRT:utility.obj
 0001:00008830       ___scrt_dllmain_exception_filter 10009830 f   MSVCRT:utility.obj
 0001:00008864       ___scrt_dllmain_uninitialize_c 10009864 f   MSVCRT:utility.obj
 0001:00008887       ___scrt_dllmain_uninitialize_critical 10009887 f   MSVCRT:utility.obj
 0001:00008894       ___scrt_initialize_crt     10009894 f   MSVCRT:utility.obj
 0001:000088cd       ___scrt_initialize_onexit_tables 100098cd f   MSVCRT:utility.obj
 0001:00008954       ___scrt_is_nonwritable_in_current_image 10009954 f   MSVCRT:utility.obj
 0001:000089e8       ___scrt_release_startup_lock 100099e8 f   MSVCRT:utility.obj
 0001:00008a05       ___scrt_uninitialize_crt   10009a05 f   MSVCRT:utility.obj
 0001:00008a2d       ___scrt_get_dyn_tls_init_callback 10009a2d f   MSVCRT:dyn_tls_init.obj
 0001:00008a33       ___scrt_fastfail           10009a33 f   MSVCRT:utility_desktop.obj
 0001:00008b4e       __crt_debugger_hook        10009b4e f   MSVCRT:utility_desktop.obj
 0001:00008b56       __RTC_Initialize           10009b56 f   MSVCRT:initsect.obj
 0001:00008b82       __RTC_Terminate            10009b82 f   MSVCRT:initsect.obj
 0001:00008bb0       __SEH_prolog4              10009bb0 f   MSVCRT:sehprolg4.obj
 0001:00008bf5       __except_handler4          10009bf5 f   MSVCRT:chandler4gs.obj
 0001:00008c24       @_guard_check_icall_nop@4  10009c24 f i MSVCRT:guard_support.obj
 0001:00008c27       ___isa_available_init      10009c27 f   MSVCRT:cpu_disp.obj
 0001:00008dfb       __get_startup_argv_mode    10009dfb f   MSVCRT:argv_mode.obj
 0001:00008dff       ___scrt_is_ucrt_dll_in_use 10009dff f   MSVCRT:ucrt_detection.obj
 0001:00008e0b       _memcpy                    10009e0b f   vcruntime:VCRUNTIME140.dll
 0001:00008e11       _memset                    10009e11 f   vcruntime:VCRUNTIME140.dll
 0001:00008e17       ___std_type_info_destroy_list 10009e17 f   vcruntime:VCRUNTIME140.dll
 0001:00008e1d       __except_handler4_common   10009e1d f   vcruntime:VCRUNTIME140.dll
 0001:00008e23       _strcmp                    10009e23 f   ucrt:api-ms-win-crt-string-l1-1-0.dll
 0001:00008e29       _strcat                    10009e29 f   ucrt:api-ms-win-crt-string-l1-1-0.dll
 0001:00008e2f       _strcpy                    10009e2f f   ucrt:api-ms-win-crt-string-l1-1-0.dll
 0001:00008e35       _strlen                    10009e35 f   ucrt:api-ms-win-crt-string-l1-1-0.dll
 0001:00008e3b       __initterm                 10009e3b f   ucrt:api-ms-win-crt-runtime-l1-1-0.dll
 0001:00008e41       __initterm_e               10009e41 f   ucrt:api-ms-win-crt-runtime-l1-1-0.dll
 0001:00008e47       __seh_filter_dll           10009e47 f   ucrt:api-ms-win-crt-runtime-l1-1-0.dll
 0001:00008e4d       __configure_narrow_argv    10009e4d f   ucrt:api-ms-win-crt-runtime-l1-1-0.dll
 0001:00008e53       __initialize_narrow_environment 10009e53 f   ucrt:api-ms-win-crt-runtime-l1-1-0.dll
 0001:00008e59       __initialize_onexit_table  10009e59 f   ucrt:api-ms-win-crt-runtime-l1-1-0.dll
 0001:00008e5f       __execute_onexit_table     10009e5f f   ucrt:api-ms-win-crt-runtime-l1-1-0.dll
 0001:00008e65       __cexit                    10009e65 f   ucrt:api-ms-win-crt-runtime-l1-1-0.dll
 0001:00008e6b       ___acrt_initialize         10009e6b f   MSVCRT:ucrt_stubs.obj
 0001:00008e6b       ___acrt_thread_attach      10009e6b f   MSVCRT:ucrt_stubs.obj
 0001:00008e6b       ___acrt_thread_detach      10009e6b f   MSVCRT:ucrt_stubs.obj
 0001:00008e6b       ___acrt_uninitialize       10009e6b f   MSVCRT:ucrt_stubs.obj
 0001:00008e6b       ___acrt_uninitialize_critical 10009e6b f   MSVCRT:ucrt_stubs.obj
 0001:00008e6b       ___scrt_stub_for_acrt_initialize 10009e6b f   MSVCRT:ucrt_stubs.obj
 0001:00008e6b       ___scrt_stub_for_acrt_thread_attach 10009e6b f   MSVCRT:ucrt_stubs.obj
 0001:00008e6b       ___scrt_stub_for_acrt_thread_detach 10009e6b f   MSVCRT:ucrt_stubs.obj
 0001:00008e6b       ___scrt_stub_for_acrt_uninitialize 10009e6b f   MSVCRT:ucrt_stubs.obj
 0001:00008e6b       ___scrt_stub_for_acrt_uninitialize_critical 10009e6b f   MSVCRT:ucrt_stubs.obj
 0001:00008e6b       ___vcrt_initialize         10009e6b f   MSVCRT:ucrt_stubs.obj
 0001:00008e6b       ___vcrt_thread_attach      10009e6b f   MSVCRT:ucrt_stubs.obj
 0001:00008e6b       ___vcrt_thread_detach      10009e6b f   MSVCRT:ucrt_stubs.obj
 0001:00008e6b       ___vcrt_uninitialize       10009e6b f   MSVCRT:ucrt_stubs.obj
 0001:00008e6b       ___vcrt_uninitialize_critical 10009e6b f   MSVCRT:ucrt_stubs.obj
 0001:00008e6e       ___scrt_stub_for_is_c_termination_complete 10009e6e f   MSVCRT:ucrt_stubs.obj
 0001:00008e6e       __is_c_termination_complete 10009e6e f   MSVCRT:ucrt_stubs.obj
 0001:00008e71       __filter_x86_sse2_floating_point_exception 10009e71 f   MSVCRT:x86_exception_filter.obj
 0001:00008e71       __filter_x86_sse2_floating_point_exception_default 10009e71 f   MSVCRT:x86_exception_filter.obj
 0002:00000000       __imp__GetLastError@0      1000a000     kernel32:KERNEL32.dll
 0002:00000004       __imp__GetModuleHandleA@4  1000a004     kernel32:KERNEL32.dll
 0002:00000008       __imp__GetProcAddress@8    1000a008     kernel32:KERNEL32.dll
 0002:0000000c       __imp__LoadLibraryA@4      1000a00c     kernel32:KERNEL32.dll
 0002:00000010       __imp__LocalFree@4         1000a010     kernel32:KERNEL32.dll
 0002:00000014       __imp__FormatMessageA@28   1000a014     kernel32:KERNEL32.dll
 0002:00000018       __imp__FreeLibrary@4       1000a018     kernel32:KERNEL32.dll
 0002:0000001c       __imp__UnhandledExceptionFilter@4 1000a01c     kernel32:KERNEL32.dll
 0002:00000020       __imp__SetUnhandledExceptionFilter@4 1000a020     kernel32:KERNEL32.dll
 0002:00000024       __imp__GetCurrentProcess@0 1000a024     kernel32:KERNEL32.dll
 0002:00000028       __imp__TerminateProcess@8  1000a028     kernel32:KERNEL32.dll
 0002:0000002c       __imp__IsProcessorFeaturePresent@4 1000a02c     kernel32:KERNEL32.dll
 0002:00000030       __imp__QueryPerformanceCounter@4 1000a030     kernel32:KERNEL32.dll
 0002:00000034       __imp__GetCurrentProcessId@0 1000a034     kernel32:KERNEL32.dll
 0002:00000038       __imp__GetCurrentThreadId@0 1000a038     kernel32:KERNEL32.dll
 0002:0000003c       __imp__GetSystemTimeAsFileTime@4 1000a03c     kernel32:KERNEL32.dll
 0002:00000040       __imp__DisableThreadLibraryCalls@4 1000a040     kernel32:KERNEL32.dll
 0002:00000044       __imp__InitializeSListHead@4 1000a044     kernel32:KERNEL32.dll
 0002:00000048       __imp__IsDebuggerPresent@0 1000a048     kernel32:KERNEL32.dll
 0002:0000004c       \177KERNEL32_NULL_THUNK_DATA 1000a04c     kernel32:KERNEL32.dll
 0002:00000050       __imp__memset              1000a050     vcruntime:VCRUNTIME140.dll
 0002:00000054       __imp____std_type_info_destroy_list 1000a054     vcruntime:VCRUNTIME140.dll
 0002:00000058       __imp___except_handler4_common 1000a058     vcruntime:VCRUNTIME140.dll
 0002:0000005c       __imp__memcpy              1000a05c     vcruntime:VCRUNTIME140.dll
 0002:00000060       \177VCRUNTIME140_NULL_THUNK_DATA 1000a060     vcruntime:VCRUNTIME140.dll
 0002:00000064       __imp__calloc              1000a064     ucrt:api-ms-win-crt-heap-l1-1-0.dll
 0002:00000068       __imp__free                1000a068     ucrt:api-ms-win-crt-heap-l1-1-0.dll
 0002:0000006c       __imp__malloc              1000a06c     ucrt:api-ms-win-crt-heap-l1-1-0.dll
 0002:00000070       \177api-ms-win-crt-heap-l1-1-0_NULL_THUNK_DATA 1000a070     ucrt:api-ms-win-crt-heap-l1-1-0.dll
 0002:00000074       __imp___seh_filter_dll     1000a074     ucrt:api-ms-win-crt-runtime-l1-1-0.dll
 0002:00000078       __imp___cexit              1000a078     ucrt:api-ms-win-crt-runtime-l1-1-0.dll
 0002:0000007c       __imp___execute_onexit_table 1000a07c     ucrt:api-ms-win-crt-runtime-l1-1-0.dll
 0002:00000080       __imp___initialize_onexit_table 1000a080     ucrt:api-ms-win-crt-runtime-l1-1-0.dll
 0002:00000084       __imp___initterm           1000a084     ucrt:api-ms-win-crt-runtime-l1-1-0.dll
 0002:00000088       __imp___initterm_e         1000a088     ucrt:api-ms-win-crt-runtime-l1-1-0.dll
 0002:0000008c       __imp___configure_narrow_argv 1000a08c     ucrt:api-ms-win-crt-runtime-l1-1-0.dll
 0002:00000090       __imp___initialize_narrow_environment 1000a090     ucrt:api-ms-win-crt-runtime-l1-1-0.dll
 0002:00000094       \177api-ms-win-crt-runtime-l1-1-0_NULL_THUNK_DATA 1000a094     ucrt:api-ms-win-crt-runtime-l1-1-0.dll
 0002:00000098       __imp__fflush              1000a098     ucrt:api-ms-win-crt-stdio-l1-1-0.dll
 0002:0000009c       __imp____acrt_iob_func     1000a09c     ucrt:api-ms-win-crt-stdio-l1-1-0.dll
 0002:000000a0       __imp____stdio_common_vsprintf 1000a0a0     ucrt:api-ms-win-crt-stdio-l1-1-0.dll
 0002:000000a4       __imp____stdio_common_vfprintf 1000a0a4     ucrt:api-ms-win-crt-stdio-l1-1-0.dll
 0002:000000a8       \177api-ms-win-crt-stdio-l1-1-0_NULL_THUNK_DATA 1000a0a8     ucrt:api-ms-win-crt-stdio-l1-1-0.dll
 0002:000000ac       __imp__strlen              1000a0ac     ucrt:api-ms-win-crt-string-l1-1-0.dll
 0002:000000b0       __imp__strncmp             1000a0b0     ucrt:api-ms-win-crt-string-l1-1-0.dll
 0002:000000b4       __imp__strcpy              1000a0b4     ucrt:api-ms-win-crt-string-l1-1-0.dll
 0002:000000b8       __imp__strcat              1000a0b8     ucrt:api-ms-win-crt-string-l1-1-0.dll
 0002:000000bc       __imp__strcmp              1000a0bc     ucrt:api-ms-win-crt-string-l1-1-0.dll
 0002:000000c0       \177api-ms-win-crt-string-l1-1-0_NULL_THUNK_DATA 1000a0c0     ucrt:api-ms-win-crt-string-l1-1-0.dll
 0002:000000c4       ___guard_check_icall_fptr  1000a0c4     MSVCRT:guard_support.obj
 0002:000000c8       ___castguard_check_failure_os_handled_fptr 1000a0c8     MSVCRT:guard_support.obj
 0002:000000cc       ___xc_a                    1000a0cc     MSVCRT:initializers.obj
 0002:000000d0       ___xc_z                    1000a0d0     MSVCRT:initializers.obj
 0002:000000d4       ___xi_a                    1000a0d4     MSVCRT:initializers.obj
 0002:000000d8       ___xi_z                    1000a0d8     MSVCRT:initializers.obj
 0002:000000dc       ___xp_a                    1000a0dc     MSVCRT:initializers.obj
 0002:000000e0       ___xp_z                    1000a0e0     MSVCRT:initializers.obj
 0002:000000e4       ___xt_a                    1000a0e4     MSVCRT:initializers.obj
 0002:000000e8       ___xt_z                    1000a0e8     MSVCRT:initializers.obj
 0002:000000f0       ??_C@_0BB@EFFKAOLB@NSS_VersionCheck@ 1000a0f0     j2secmod.obj
 0002:00000104       ??_C@_0P@JCBGNBMA@NSS_Initialize@ 1000a104     j2secmod.obj
 0002:00000114       ??_C@_09GOBCDJFC@secmod?4db@ 1000a114     j2secmod.obj
 0002:00000120       ??_C@_04DAEILJDJ@sql?3@    1000a120     j2secmod.obj
 0002:00000128       ??_C@_0L@EOEDJBCP@pkcs11?4txt@ 1000a128     j2secmod.obj
 0002:00000134       ??_C@_08LJKFHILM@NSS_Init@ 1000a134     j2secmod.obj
 0002:0000013d       ??_C@_00CNPNBAHC@@         1000a13d     j2secmod.obj
 0002:00000140       ??_C@_0BC@KONLDBJC@NSS_InitReadWrite@ 1000a140     j2secmod.obj
 0002:00000154       ??_C@_0O@LCPIEDLO@NSS_NoDB_Init@ 1000a154     j2secmod.obj
 0002:00000164       ??_C@_0BM@FOILBMDH@SECMOD_GetDefaultModuleList@ 1000a164     j2secmod.obj
 0002:00000180       ??_C@_0BE@GPOIDJOH@java?1util?1ArrayList@ 1000a180     j2secmod.obj
 0002:00000194       ??_C@_03GAEACAIP@?$CI?$CJV@ 1000a194     j2secmod.obj
 0002:00000198       ??_C@_06FALKBLGB@?$DMinit?$DO@ 1000a198     j2secmod.obj
 0002:000001a0       ??_C@_0BG@DHOOFEJE@?$CILjava?1lang?1Object?$DL?$CJZ@ 1000a1a0     j2secmod.obj
 0002:000001b8       ??_C@_03BDGOHNNK@add@      1000a1b8     j2secmod.obj
 0002:000001bc       ??_C@_0CC@KDFBHMNN@sun?1security?1pkcs11?1Secmod$Modu@ 1000a1bc     j2secmod.obj
 0002:000001e0       ??_C@_0DM@JNKODIFA@?$CILjava?1lang?1String?$DLLjava?1lang?1S@ 1000a1e0     j2secmod.obj
 0002:0000021c       ??_C@_0BF@BNLKGCGH@Symbol?5not?5found?3?5?$CFs@ 1000a21c     j2secmod_md.obj
 0002:00000234       ??_C@_0CE@BDNBALGO@sun?1security?1pkcs11?1wrapper?1CK_@ 1000a234     p11_convert.obj
 0002:00000258       ??_C@_09KCOLIFDD@?$CI?$FLC?$FLC?$FLC?$CJV@ 1000a258     p11_convert.obj
 0002:00000264       ??_C@_0CH@FAGBPBAL@sun?1security?1pkcs11?1wrapper?1CK_@ 1000a264     p11_convert.obj
 0002:0000028c       ??_C@_05MNEAHDDF@?$CIII?$CJV@ 1000a28c     p11_convert.obj
 0002:00000294       ??_C@_0CM@LGADNNOP@sun?1security?1pkcs11?1wrapper?1CK_@ 1000a294     p11_convert.obj
 0002:000002c0       ??_C@_07MDGBCFEE@?$CIJJJJ?$CJV@ 1000a2c0     p11_convert.obj
 0002:000002c8       ??_C@_0CJ@KOKMKMLD@sun?1security?1pkcs11?1wrapper?1CK_@ 1000a2c8     p11_convert.obj
 0002:000002f4       ??_C@_0BH@CPAPLJAG@?$CIJLjava?1lang?1Object?$DL?$CJV@ 1000a2f4     p11_convert.obj
 0002:0000030c       ??_C@_01HMGJMAIH@B@        1000a30c     p11_convert.obj
 0002:00000310       ??_C@_05FEBMJMCL@major@    1000a310     p11_convert.obj
 0002:00000318       ??_C@_05OLAOEALN@minor@    1000a318     p11_convert.obj
 0002:00000320       ??_C@_02LLADPLHK@?$FLC@    1000a320     p11_convert.obj
 0002:00000324       ??_C@_04JFPLDHAO@year@     1000a324     p11_convert.obj
 0002:0000032c       ??_C@_05MEBAADFH@month@    1000a32c     p11_convert.obj
 0002:00000334       ??_C@_03NNBHCDBP@day@      1000a334     p11_convert.obj
 0002:00000338       ??_C@_01LELAEKIP@J@        1000a338     p11_convert.obj
 0002:0000033c       ??_C@_04GPMDFGEJ@type@     1000a33c     p11_convert.obj
 0002:00000344       ??_C@_0BD@HMGGFBMH@Ljava?1lang?1Object?$DL@ 1000a344     p11_convert.obj
 0002:00000358       ??_C@_06MLDODIFP@pValue@   1000a358     p11_convert.obj
 0002:00000360       ??_C@_0DC@HGPFDFFP@Lsun?1security?1pkcs11?1wrapper?1CK@ 1000a360     p11_convert.obj
 0002:00000394       ??_C@_0L@KDDOOLLF@RandomInfo@ 1000a394     p11_convert.obj
 0002:000003a0       ??_C@_0DA@MGBKDFKC@sun?1security?1pkcs11?1wrapper?1CK_@ 1000a3a0     p11_convert.obj
 0002:000003d0       ??_C@_02KCBIMKDL@?$FLB@    1000a3d0     p11_convert.obj
 0002:000003d4       ??_C@_0O@DPKEFPKK@pClientRandom@ 1000a3d4     p11_convert.obj
 0002:000003e4       ??_C@_0O@BDHOCNNP@pServerRandom@ 1000a3e4     p11_convert.obj
 0002:000003f4       ??_C@_0CJ@KHCANOHB@Lsun?1security?1pkcs11?1wrapper?1CK@ 1000a3f4     p11_convert.obj
 0002:00000420       ??_C@_08KFNBPFOP@pVersion@ 1000a420     p11_convert.obj
 0002:0000042c       ??_C@_0DN@HBKDAKMN@sun?1security?1pkcs11?1wrapper?1CK_@ 1000a42c     p11_convert.obj
 0002:0000046c       ??_C@_0DO@JGMPNKLG@sun?1security?1pkcs11?1wrapper?1CK_@ 1000a46c     p11_convert.obj
 0002:000004ac       ??_C@_0BB@MMANIKKH@prfHashMechanism@ 1000a4ac     p11_convert.obj
 0002:000004c0       ??_C@_0CO@DCJBCFCB@sun?1security?1pkcs11?1wrapper?1CK_@ 1000a4c0     p11_convert.obj
 0002:000004f0       ??_C@_05HJNJEGNP@pSeed@    1000a4f0     p11_convert.obj
 0002:000004f8       ??_C@_06EEEIHGKI@pLabel@   1000a4f8     p11_convert.obj
 0002:00000500       ??_C@_07KBCFNIDO@pOutput@  1000a500     p11_convert.obj
 0002:00000508       ??_C@_0CO@NBPNNDEJ@sun?1security?1pkcs11?1wrapper?1CK_@ 1000a508     p11_convert.obj
 0002:00000538       ??_C@_0N@IEICAFHB@prfMechanism@ 1000a538     p11_convert.obj
 0002:00000548       ??_C@_0M@LJIINDHF@ulMacLength@ 1000a548     p11_convert.obj
 0002:00000554       ??_C@_0BB@BJFICNNC@ulServerOrClient@ 1000a554     p11_convert.obj
 0002:00000568       ??_C@_0BA@CKOIHILJ@ulMacSizeInBits@ 1000a568     p11_convert.obj
 0002:00000578       ??_C@_0BA@PELMFMAE@ulKeySizeInBits@ 1000a578     p11_convert.obj
 0002:00000588       ??_C@_0P@LDDDJGAG@ulIVSizeInBits@ 1000a588     p11_convert.obj
 0002:00000598       ??_C@_01POHCFINO@Z@        1000a598     p11_convert.obj
 0002:0000059c       ??_C@_09OOHKLCMP@bIsExport@ 1000a59c     p11_convert.obj
 0002:000005a8       ??_C@_0DA@CCEPBHDJ@sun?1security?1pkcs11?1wrapper?1CK_@ 1000a5a8     p11_convert.obj
 0002:000005d8       ??_C@_0DC@BBMMCKLB@Lsun?1security?1pkcs11?1wrapper?1CK@ 1000a5d8     p11_convert.obj
 0002:0000060c       ??_C@_0BF@ODGIPGLB@pReturnedKeyMaterial@ 1000a60c     p11_convert.obj
 0002:00000624       ??_C@_09JAFBLFBM@pIVClient@ 1000a624     p11_convert.obj
 0002:00000630       ??_C@_09NPBDGOJP@pIVServer@ 1000a630     p11_convert.obj
 0002:0000063c       ??_C@_0DD@IELHHAPM@sun?1security?1pkcs11?1wrapper?1CK_@ 1000a63c     p11_convert.obj
 0002:00000670       ??_C@_0DE@JIDMGMIB@sun?1security?1pkcs11?1wrapper?1CK_@ 1000a670     p11_convert.obj
 0002:000006a4       ??_C@_0CO@CAAEDKFF@sun?1security?1pkcs11?1wrapper?1CK_@ 1000a6a4     p11_convert.obj
 0002:000006d4       ??_C@_0O@FAFICCFK@ulCounterBits@ 1000a6d4     p11_convert.obj
 0002:000006e4       ??_C@_02BNOEFKLB@cb@       1000a6e4     p11_convert.obj
 0002:000006e8       ??_C@_0CK@NKNHHAJC@sun?1security?1pkcs11?1wrapper?1CK_@ 1000a6e8     p11_convert.obj
 0002:00000714       ??_C@_02DONNAIDC@iv@       1000a714     p11_convert.obj
 0002:00000718       ??_C@_03BFKFLPDB@aad@      1000a718     p11_convert.obj
 0002:0000071c       ??_C@_07LJAAJOFG@tagBits@  1000a71c     p11_convert.obj
 0002:00000724       ??_C@_0CK@GKAOADBA@sun?1security?1pkcs11?1wrapper?1CK_@ 1000a724     p11_convert.obj
 0002:00000750       ??_C@_07LDPMHAML@dataLen@  1000a750     p11_convert.obj
 0002:00000758       ??_C@_05OOEDLKEB@nonce@    1000a758     p11_convert.obj
 0002:00000760       ??_C@_06PBGIHEKB@macLen@   1000a760     p11_convert.obj
 0002:00000768       ??_C@_0EA@NNBELOMA@sun?1security?1pkcs11?1wrapper?1CK_@ 1000a768     p11_convert.obj
 0002:000007a8       ??_C@_0CI@ELKCPMM@No?5parameter?5support?5for?5this?5m@ 1000a7a8     p11_convert.obj
 0002:000007d0       ??_C@_0DE@FNJOAKHM@sun?1security?1pkcs11?1wrapper?1CK_@ 1000a7d0     p11_convert.obj
 0002:00000804       ??_C@_07NIDPGPFG@hashAlg@  1000a804     p11_convert.obj
 0002:0000080c       ??_C@_03GJMIBOLJ@mgf@      1000a80c     p11_convert.obj
 0002:00000810       ??_C@_06OEKOLKIL@source@   1000a810     p11_convert.obj
 0002:00000818       ??_C@_0M@NGABHANP@pSourceData@ 1000a818     p11_convert.obj
 0002:00000824       ??_C@_0CK@JAAGIPM@sun?1security?1pkcs11?1wrapper?1CK_@ 1000a824     p11_convert.obj
 0002:00000850       ??_C@_0M@GGOAOMAD@pInitVector@ 1000a850     p11_convert.obj
 0002:0000085c       ??_C@_09KKEKIPIM@pPassword@ 1000a85c     p11_convert.obj
 0002:00000868       ??_C@_05LDKIPIFG@pSalt@    1000a868     p11_convert.obj
 0002:00000870       ??_C@_0M@HPDAPCKI@ulIteration@ 1000a870     p11_convert.obj
 0002:0000087c       ??_C@_0CJ@EEABPKHL@sun?1security?1pkcs11?1wrapper?1CK_@ 1000a87c     p11_convert.obj
 0002:000008a8       ??_C@_09ONMFBHMB@mechanism@ 1000a8a8     p11_convert.obj
 0002:000008b4       ??_C@_0L@JBCBPDO@pParameter@ 1000a8b4     p11_convert.obj
 0002:000008c0       ??_C@_0M@FGJAKHMC@pInitVektor@ 1000a8c0     p11_convert.obj
 0002:000008cc       ??_C@_0DC@OALCDCIB@sun?1security?1pkcs11?1wrapper?1CK_@ 1000a8cc     p11_convert.obj
 0002:00000900       ??_C@_0L@BGFAFLOD@saltSource@ 1000a900     p11_convert.obj
 0002:0000090c       ??_C@_0BA@IHHAPGDC@pSaltSourceData@ 1000a90c     p11_convert.obj
 0002:0000091c       ??_C@_0L@LEIMKHLK@iterations@ 1000a91c     p11_convert.obj
 0002:00000928       ??_C@_03NBFGPAGA@prf@      1000a928     p11_convert.obj
 0002:0000092c       ??_C@_08BINOACIC@pPrfData@ 1000a92c     p11_convert.obj
 0002:00000938       ??_C@_0DD@JKKJEEHE@sun?1security?1pkcs11?1wrapper?1CK_@ 1000a938     p11_convert.obj
 0002:0000096c       ??_C@_04ODAPDKJK@sLen@     1000a96c     p11_convert.obj
 0002:00000974       ??_C@_0DD@BKPMIPL@sun?1security?1pkcs11?1wrapper?1CK_@ 1000a974     p11_convert.obj
 0002:000009a8       ??_C@_03EOOFPPDM@kdf@      1000a9a8     p11_convert.obj
 0002:000009ac       ??_C@_0M@GNHNJOEE@pSharedData@ 1000a9ac     p11_convert.obj
 0002:000009b8       ??_C@_0M@KMNGLHAN@pPublicData@ 1000a9b8     p11_convert.obj
 0002:000009c4       ??_C@_0DD@CIGHHMAJ@sun?1security?1pkcs11?1wrapper?1CK_@ 1000a9c4     p11_convert.obj
 0002:000009f8       ??_C@_0BB@FHLLIPHA@ulPrivateDataLen@ 1000a9f8     p11_convert.obj
 0002:00000a0c       ??_C@_0N@MNKNKKOE@hPrivateData@ 1000aa0c     p11_convert.obj
 0002:00000a1c       ??_C@_0N@JDGNPOHL@pPublicData2@ 1000aa1c     p11_convert.obj
 0002:00000a2c       ??_C@_0DH@KLOKCPBP@sun?1security?1pkcs11?1wrapper?1CK_@ 1000aa2c     p11_convert.obj
 0002:00000a64       ??_C@_0L@BEOLNMGA@pOtherInfo@ 1000aa64     p11_convert.obj
 0002:00000a70       ??_C@_0DH@ICCCJLON@sun?1security?1pkcs11?1wrapper?1CK_@ 1000aa70     p11_convert.obj
 0002:00000aa8       ??_C@_0M@KOOGEDPH@pNativeData@ 1000aaa8     p11_general.obj
 0002:00000ab4       ??_C@_07EJMAFCDJ@pHandle@  1000aab4     p11_general.obj
 0002:00000abc       ??_C@_0P@MLLHBNNC@java?1lang?1Long@ 1000aabc     p11_general.obj
 0002:00000acc       ??_C@_0CE@FGGPEABN@sun?1security?1pkcs11?1wrapper?1CK_@ 1000aacc     p11_general.obj
 0002:00000af0       ??_C@_0FJ@PCBLKCL@?$CILsun?1security?1pkcs11?1wrapper?1C@ 1000aaf0     p11_general.obj
 0002:00000b4c       ??_C@_0CJ@BIOEJKNF@sun?1security?1pkcs11?1wrapper?1CK_@ 1000ab4c     p11_general.obj
 0002:00000b78       ??_C@_0FJ@OBILFDMI@?$CI?$FLC?$FLCJLsun?1security?1pkcs11?1wrap@ 1000ab78     p11_general.obj
 0002:00000bd4       ??_C@_0CK@MCNCOGLO@sun?1security?1pkcs11?1wrapper?1CK_@ 1000abd4     p11_general.obj
 0002:00000c00       ??_C@_0GJ@FDGHLOMM@?$CI?$FLC?$FLC?$FLC?$FLCJJJJJJJJJJJLsun?1securi@ 1000ac00     p11_general.obj
 0002:00000c6c       ??_C@_0CO@CCAIMKIH@sun?1security?1pkcs11?1wrapper?1CK_@ 1000ac6c     p11_general.obj
 0002:00000c9c       ??_C@_06NJFABHM@?$CIJJJ?$CJV@ 1000ac9c     p11_general.obj
 0002:00000ca8       ??_C@_0HA@JHHDDDM@C_1GenerateKeyPair?$CI?$CJ?3?5C_Generat@ 1000aca8     p11_keymgmt.obj
 0002:00000d18       ??_C@_0BB@DDIADMEB@hClientMacSecret@ 1000ad18     p11_keymgmt.obj
 0002:00000d2c       ??_C@_0BB@BKLFLGGI@hServerMacSecret@ 1000ad2c     p11_keymgmt.obj
 0002:00000d40       ??_C@_0L@GFMHBDMC@hClientKey@ 1000ad40     p11_keymgmt.obj
 0002:00000d4c       ??_C@_0L@HMKKIKDM@hServerKey@ 1000ad4c     p11_keymgmt.obj
 0002:00000d58       ??_C@_0DB@KELDKOFM@sun?1security?1pkcs11?1wrapper?1CK_@ 1000ad58     p11_mutex.obj
 0002:00000d8c       ??_C@_0CN@MIBMAGA@Lsun?1security?1pkcs11?1wrapper?1CK@ 1000ad8c     p11_mutex.obj
 0002:00000dbc       ??_C@_0M@CHIIKKKK@CreateMutex@ 1000adbc     p11_mutex.obj
 0002:00000dc8       ??_C@_0CO@KLPPKFHK@Lsun?1security?1pkcs11?1wrapper?1CK@ 1000adc8     p11_mutex.obj
 0002:00000df8       ??_C@_0N@MEBBDPAH@DestroyMutex@ 1000adf8     p11_mutex.obj
 0002:00000e08       ??_C@_0CL@LBHOKNDM@Lsun?1security?1pkcs11?1wrapper?1CK@ 1000ae08     p11_mutex.obj
 0002:00000e34       ??_C@_09DKPDKGG@LockMutex@ 1000ae34     p11_mutex.obj
 0002:00000e40       ??_C@_0CN@KJNOCKKG@Lsun?1security?1pkcs11?1wrapper?1CK@ 1000ae40     p11_mutex.obj
 0002:00000e70       ??_C@_0M@HCNHAHIN@UnlockMutex@ 1000ae70     p11_mutex.obj
 0002:00000e7c       ??_C@_05GECEPKB@flags@     1000ae7c     p11_mutex.obj
 0002:00000e84       ??_C@_09CJOBGKOG@pReserved@ 1000ae84     p11_mutex.obj
 0002:00000e90       ??_C@_0CL@FFENGHBF@sun?1security?1pkcs11?1wrapper?1CK_@ 1000ae90     p11_mutex.obj
 0002:00000ebc       ??_C@_0BF@LHBAMMHC@?$CI?$CJLjava?1lang?1Object?$DL@ 1000aebc     p11_mutex.obj
 0002:00000ed4       ??_C@_0P@MBLCOHGI@CK_CREATEMUTEX@ 1000aed4     p11_mutex.obj
 0002:00000ee4       ??_C@_0CM@EDGLGECO@sun?1security?1pkcs11?1wrapper?1PKC@ 1000aee4     p11_mutex.obj
 0002:00000f10       ??_C@_03IGDHHNNC@?$CI?$CJJ@ 1000af10     p11_mutex.obj
 0002:00000f14       ??_C@_0N@CFOEEHFM@getErrorCode@ 1000af14     p11_mutex.obj
 0002:00000f24       ??_C@_0CM@MCCIEMNP@sun?1security?1pkcs11?1wrapper?1CK_@ 1000af24     p11_mutex.obj
 0002:00000f50       ??_C@_0BG@JLFLBLJI@?$CILjava?1lang?1Object?$DL?$CJV@ 1000af50     p11_mutex.obj
 0002:00000f68       ??_C@_0BA@OMAILONO@CK_DESTROYMUTEX@ 1000af68     p11_mutex.obj
 0002:00000f78       ??_C@_0CJ@OCJKNBDK@sun?1security?1pkcs11?1wrapper?1CK_@ 1000af78     p11_mutex.obj
 0002:00000fa4       ??_C@_0N@DNKBOIPK@CK_LOCKMUTEX@ 1000afa4     p11_mutex.obj
 0002:00000fb4       ??_C@_0CL@BCMKDC@sun?1security?1pkcs11?1wrapper?1CK_@ 1000afb4     p11_mutex.obj
 0002:00000fe0       ??_C@_0P@JEONEKEP@CK_UNLOCKMUTEX@ 1000afe0     p11_mutex.obj
 0002:00000ff0       ??_C@_06MELFAPKK@?50x?$CFlX@ 1000aff0     p11_objmgmt.obj
 0002:00000ff8       ??_C@_0CG@KHGOBKJJ@sun?1security?1pkcs11?1wrapper?1CK_@ 1000aff8     p11_sessmgmt.obj
 0002:00001020       ??_C@_0BI@DIAMFDOH@?$CIJJLjava?1lang?1Object?$DL?$CJV@ 1000b020     p11_sessmgmt.obj
 0002:00001038       ??_C@_09GHOCIINE@CK_NOTIFY@ 1000b038     p11_sessmgmt.obj
 0002:00001044       ??_C@_0BB@DDFKOHA@java?1lang?1Object@ 1000b044     p11_util.obj
 0002:00001058       ??_C@_0BH@DOGHFNPN@?$CIJLjava?1lang?1String?$DL?$CJV@ 1000b058     p11_util.obj
 0002:00001070       ??_C@_0BL@ENCPOIKC@java?1lang?1OutOfMemoryError@ 1000b070     p11_util.obj
 0002:0000108c       ??_C@_0BP@GJLHLAKJ@java?1lang?1NullPointerException@ 1000b08c     p11_util.obj
 0002:000010ac       ??_C@_0BE@EBAPEBGJ@java?1io?1IOException@ 1000b0ac     p11_util.obj
 0002:000010c0       ??_C@_0DD@DEDAKGI@sun?1security?1pkcs11?1wrapper?1PKC@ 1000b0c0     p11_util.obj
 0002:000010f4       ??_C@_0CK@GAEPNKCI@This?5object?5is?5not?5connected?5to@ 1000b0f4     p11_util.obj
 0002:00001120       ??_C@_0BC@DDPBLLCP@java?1lang?1Boolean@ 1000b120     p11_util.obj
 0002:00001134       ??_C@_04LHKBAEFM@?$CIZ?$CJV@ 1000b134     p11_util.obj
 0002:0000113c       ??_C@_04OHLIFDMD@?$CIJ?$CJV@ 1000b13c     p11_util.obj
 0002:00001144       ??_C@_03MMPFGPID@?$CI?$CJZ@ 1000b144     p11_util.obj
 0002:00001148       ??_C@_0N@FIOMDIJC@booleanValue@ 1000b148     p11_util.obj
 0002:00001158       ??_C@_0P@CCHCOPNE@java?1lang?1Byte@ 1000b158     p11_util.obj
 0002:00001168       ??_C@_03EOOOPHNK@?$CI?$CJB@ 1000b168     p11_util.obj
 0002:0000116c       ??_C@_09CBDGACJH@byteValue@ 1000b16c     p11_util.obj
 0002:00001178       ??_C@_0BC@OHJKABOO@java?1lang?1Integer@ 1000b178     p11_util.obj
 0002:0000118c       ??_C@_03KNBKCOBB@?$CI?$CJI@ 1000b18c     p11_util.obj
 0002:00001190       ??_C@_08HBLFFCOK@intValue@ 1000b190     p11_util.obj
 0002:0000119c       ??_C@_09JKMBDFBF@longValue@ 1000b19c     p11_util.obj
 0002:000011a8       ??_C@_0P@OINJBDJD@java?1lang?1Char@ 1000b1a8     p11_util.obj
 0002:000011b8       ??_C@_03FHPFMGJL@?$CI?$CJC@ 1000b1b8     p11_util.obj
 0002:000011bc       ??_C@_09ODGNKCJE@charValue@ 1000b1bc     p11_util.obj
 0002:000011c8       ??_C@_0BE@GKIHCGPM@java?1lang?1Character@ 1000b1c8     p11_util.obj
 0002:000011dc       ??_C@_02CAADFCGC@?$FLZ@    1000b1dc     p11_util.obj
 0002:000011e0       ??_C@_02EBOMBDPA@?$FLI@    1000b1e0     p11_util.obj
 0002:000011e4       ??_C@_02GKMBEADD@?$FLJ@    1000b1e4     p11_util.obj
 0002:000011e8       ??_C@_0BB@FLFAIHG@java?1lang?1String@ 1000b1e8     p11_util.obj
 0002:000011fc       ??_C@_0BE@IIFEGCLG@?$CI?$CJLjava?1lang?1Class?$DL@ 1000b1fc     p11_util.obj
 0002:00001210       ??_C@_08KFOJNDAP@getClass@ 1000b210     p11_util.obj
 0002:0000121c       ??_C@_0BA@JJLOPNCP@java?1lang?1Class@ 1000b21c     p11_util.obj
 0002:0000122c       ??_C@_0BF@FOHFOJOB@?$CI?$CJLjava?1lang?1String?$DL@ 1000b22c     p11_util.obj
 0002:00001244       ??_C@_07DFBCBEHO@getName@  1000b244     p11_util.obj
 0002:00001250       ??_C@_0EH@CMCPFLGF@Java?5object?5of?5this?5class?5canno@ 1000b250     p11_util.obj
 0002:00001298       ??_C@_0M@LFMBLMNP@sunpkcs11?3?5@ 1000b298     p11_util.obj
 0002:000012a4       __pDefaultRawDllMain       1000b2a4     MSVCRT:dll_dllmain.obj
 0002:000012a4       __pRawDllMain              1000b2a4     MSVCRT:dll_dllmain.obj
 0002:000012b0       __load_config_used         1000b2b0     MSVCRT:loadcfg.obj
 0002:00001400       ___safe_se_handler_table   1000b400     <linker-defined>
 0002:00001404       ___volatile_metadata       1000b404     <linker-defined>
 0002:00001708       ___rtc_iaa                 1000b708     MSVCRT:initsect.obj
 0002:0000170c       ___rtc_izz                 1000b70c     MSVCRT:initsect.obj
 0002:00001710       ___rtc_taa                 1000b710     MSVCRT:initsect.obj
 0002:00001714       ___rtc_tzz                 1000b714     MSVCRT:initsect.obj
 0002:00002a8c       __IMPORT_DESCRIPTOR_KERNEL32 1000ca8c     kernel32:KERNEL32.dll
 0002:00002aa0       __IMPORT_DESCRIPTOR_VCRUNTIME140 1000caa0     vcruntime:VCRUNTIME140.dll
 0002:00002ab4       __IMPORT_DESCRIPTOR_api-ms-win-crt-string-l1-1-0 1000cab4     ucrt:api-ms-win-crt-string-l1-1-0.dll
 0002:00002ac8       __IMPORT_DESCRIPTOR_api-ms-win-crt-stdio-l1-1-0 1000cac8     ucrt:api-ms-win-crt-stdio-l1-1-0.dll
 0002:00002adc       __IMPORT_DESCRIPTOR_api-ms-win-crt-heap-l1-1-0 1000cadc     ucrt:api-ms-win-crt-heap-l1-1-0.dll
 0002:00002af0       __IMPORT_DESCRIPTOR_api-ms-win-crt-runtime-l1-1-0 1000caf0     ucrt:api-ms-win-crt-runtime-l1-1-0.dll
 0002:00002b04       __NULL_IMPORT_DESCRIPTOR   1000cb04     kernel32:KERNEL32.dll
 0003:000002dc       ___security_cookie_complement 1000d2dc     MSVCRT:gs_cookie.obj
 0003:000002e0       ___security_cookie         1000d2e0     MSVCRT:gs_cookie.obj
 0003:000002f0       ___scrt_native_dllmain_reason 1000d2f0     MSVCRT:utility.obj
 0003:00000300       ___isa_enabled             1000d300     MSVCRT:cpu_disp.obj
 0003:00000304       ___scrt_ucrt_dll_is_in_use 1000d304     MSVCRT:ucrt_stubs.obj
 0003:00000308       _debug                     1000d308     p11_general.obj
 0003:0000030c       _jvm                       1000d30c     p11_general.obj
 0003:00000310       _notifyListHead            1000d310     p11_sessmgmt.obj
 0003:00000314       _notifyListLock            1000d314     p11_sessmgmt.obj
 0003:00000640       ?__type_info_root_node@@3U__type_info_node@@A 1000d640     MSVCRT:tncleanup.obj
 0003:00000648       ?_OptionsStorage@?1??__local_stdio_scanf_options@@9@4_KA 1000d648     MSVCRT:default_local_stdio_options.obj
 0003:00000650       ___scrt_current_native_startup_state 1000d650     MSVCRT:utility.obj
 0003:00000654       ___scrt_native_startup_lock 1000d654     MSVCRT:utility.obj
 0003:00000674       ___scrt_debugger_hook_flag 1000d674     MSVCRT:utility_desktop.obj
 0003:00000678       ___isa_available           1000d678     MSVCRT:cpu_disp.obj
 0003:0000067c       ___favor                   1000d67c     MSVCRT:cpu_disp.obj
 0003:00000680       _ckpGlobalInitArgs         1000d680     <common>
 0003:00000684       _jInitArgsObject           1000d684     <common>
 0003:00000688       _jLongClass                1000d688     <common>
 0003:0000068c       _jByteArrayClass           1000d68c     <common>
 0003:00000690       _mech_pHandleID            1000d690     <common>
 0003:00000694       _mech_pParameterID         1000d694     <common>
 0003:00000698       _mech_mechanismID          1000d698     <common>
 0003:0000069c       _pNativeDataID             1000d69c     <common>
 0003:000006a0       ?_OptionsStorage@?1??__local_stdio_printf_options@@9@9 1000d6a0     <common>
 0003:000006a8       ___dyn_tls_init_callback   1000d6a8     <common>

 entry point at        0001:0000851b

 Static symbols

 0000:ffff0000       .debug$S                   10000000     j2pkcs11.exp
 0000:ffff0000       .debug$S                   10000000     vcruntime:VCRUNTIME140.dll
 0000:ffff0000       .debug$S                   10000000     vcruntime:VCRUNTIME140.dll
 0000:ffff0000       .debug$S                   10000000     vcruntime:VCRUNTIME140.dll
 0000:ffff0000       .debug$S                   10000000     vcruntime:VCRUNTIME140.dll
 0000:ffff0000       .debug$S                   10000000     vcruntime:VCRUNTIME140.dll
 0000:ffff0000       .debug$S                   10000000     vcruntime:VCRUNTIME140.dll
 0000:ffff0000       .debug$S                   10000000     ucrt:api-ms-win-crt-heap-l1-1-0.dll
 0000:ffff0000       .debug$S                   10000000     ucrt:api-ms-win-crt-heap-l1-1-0.dll
 0000:ffff0000       .debug$S                   10000000     ucrt:api-ms-win-crt-heap-l1-1-0.dll
 0000:ffff0000       .debug$S                   10000000     ucrt:api-ms-win-crt-runtime-l1-1-0.dll
 0000:ffff0000       .debug$S                   10000000     ucrt:api-ms-win-crt-runtime-l1-1-0.dll
 0000:ffff0000       .debug$S                   10000000     ucrt:api-ms-win-crt-runtime-l1-1-0.dll
 0000:ffff0000       .debug$S                   10000000     ucrt:api-ms-win-crt-runtime-l1-1-0.dll
 0000:ffff0000       .debug$S                   10000000     ucrt:api-ms-win-crt-runtime-l1-1-0.dll
 0000:ffff0000       .debug$S                   10000000     ucrt:api-ms-win-crt-runtime-l1-1-0.dll
 0000:ffff0000       .debug$S                   10000000     ucrt:api-ms-win-crt-runtime-l1-1-0.dll
 0000:ffff0000       .debug$S                   10000000     ucrt:api-ms-win-crt-runtime-l1-1-0.dll
 0000:ffff0000       .debug$S                   10000000     ucrt:api-ms-win-crt-runtime-l1-1-0.dll
 0000:ffff0000       .debug$S                   10000000     ucrt:api-ms-win-crt-runtime-l1-1-0.dll
 0000:ffff0000       .debug$S                   10000000     ucrt:api-ms-win-crt-runtime-l1-1-0.dll
 0000:ffff0000       .debug$S                   10000000     ucrt:api-ms-win-crt-runtime-l1-1-0.dll
 0000:ffff0000       .debug$S                   10000000     ucrt:api-ms-win-crt-stdio-l1-1-0.dll
 0000:ffff0000       .debug$S                   10000000     ucrt:api-ms-win-crt-stdio-l1-1-0.dll
 0000:ffff0000       .debug$S                   10000000     ucrt:api-ms-win-crt-stdio-l1-1-0.dll
 0000:ffff0000       .debug$S                   10000000     ucrt:api-ms-win-crt-stdio-l1-1-0.dll
 0000:ffff0000       .debug$S                   10000000     ucrt:api-ms-win-crt-string-l1-1-0.dll
 0000:ffff0000       .debug$S                   10000000     ucrt:api-ms-win-crt-string-l1-1-0.dll
 0000:ffff0000       .debug$S                   10000000     ucrt:api-ms-win-crt-string-l1-1-0.dll
 0000:ffff0000       .debug$S                   10000000     ucrt:api-ms-win-crt-string-l1-1-0.dll
 0000:ffff0000       .debug$S                   10000000     ucrt:api-ms-win-crt-string-l1-1-0.dll
 0000:ffff0000       .debug$S                   10000000     kernel32:KERNEL32.dll
 0000:ffff0000       .debug$S                   10000000     kernel32:KERNEL32.dll
 0000:ffff0000       .debug$S                   10000000     kernel32:KERNEL32.dll
 0000:ffff0000       .debug$S                   10000000     kernel32:KERNEL32.dll
 0000:ffff0000       .debug$S                   10000000     kernel32:KERNEL32.dll
 0000:ffff0000       .debug$S                   10000000     kernel32:KERNEL32.dll
 0000:ffff0000       .debug$S                   10000000     kernel32:KERNEL32.dll
 0000:ffff0000       .debug$S                   10000000     kernel32:KERNEL32.dll
 0000:ffff0000       .debug$S                   10000000     kernel32:KERNEL32.dll
 0000:ffff0000       .debug$S                   10000000     kernel32:KERNEL32.dll
 0000:ffff0000       .debug$S                   10000000     kernel32:KERNEL32.dll
 0000:ffff0000       .debug$S                   10000000     kernel32:KERNEL32.dll
 0000:ffff0000       .debug$S                   10000000     kernel32:KERNEL32.dll
 0000:ffff0000       .debug$S                   10000000     kernel32:KERNEL32.dll
 0000:ffff0000       .debug$S                   10000000     kernel32:KERNEL32.dll
 0000:ffff0000       .debug$S                   10000000     kernel32:KERNEL32.dll
 0000:ffff0000       .debug$S                   10000000     kernel32:KERNEL32.dll
 0000:ffff0000       .debug$S                   10000000     kernel32:KERNEL32.dll
 0000:ffff0000       .debug$S                   10000000     kernel32:KERNEL32.dll
 0000:ffff0000       .debug$S                   10000000     kernel32:KERNEL32.dll
 0000:ffff0000       .debug$S                   10000000     kernel32:KERNEL32.dll
 0001:000006ef       $LN79                      100016ef     p11_convert.obj
 0001:00000703       $LN78                      10001703     p11_convert.obj
 0001:00000723       $LN81                      10001723     p11_convert.obj
 0001:0000072f       $LN80                      1000172f     p11_convert.obj
 0001:00004dea       _copyBackClientVersion     10005dea f   p11_keymgmt.obj
 0001:00004f11       _copyBackKeyMatParams      10005f11 f   p11_keymgmt.obj
 0001:000081b0       $$000000                   100091b0     MSVCRT:chkstk.obj
 0001:000081c4       cs10                       100091c4     MSVCRT:chkstk.obj
 0001:000081d2       cs20                       100091d2     MSVCRT:chkstk.obj
 0001:000081db       ?dllmain_crt_dispatch@@YGHQAUHINSTANCE__@@KQAX@Z 100091db f   MSVCRT:dll_dllmain.obj
 0001:0000822e       ?dllmain_crt_process_attach@@YAHQAUHINSTANCE__@@QAX@Z 1000922e f   MSVCRT:dll_dllmain.obj
 0001:00008335       ?dllmain_crt_process_detach@@YAH_N@Z 10009335 f   MSVCRT:dll_dllmain.obj
 0001:000083e5       ?dllmain_dispatch@@YAHQAUHINSTANCE__@@KQAX@Z 100093e5 f   MSVCRT:dll_dllmain.obj
 0001:000084f0       ?dllmain_raw@@YGHQAUHINSTANCE__@@KQAX@Z 100094f0 f   MSVCRT:dll_dllmain.obj
 0001:00008660       ___get_entropy             10009660 f   MSVCRT:gs_support.obj
 0001:00008755       ?find_pe_section@@YAPAU_IMAGE_SECTION_HEADER@@QAEI@Z 10009755 f   MSVCRT:utility.obj
 0001:00008bb0       $$000000                   10009bb0     MSVCRT:sehprolg4.obj
 0002:000012a8       _GS_ExceptionPointers      1000b2a8     MSVCRT:gs_report.obj
 0002:00001718       __sehtable$?dllmain_crt_process_attach@@YAHQAUHINSTANCE__@@QAX@Z 1000b718     MSVCRT:dll_dllmain.obj
 0002:00001738       __sehtable$?dllmain_crt_process_detach@@YAH_N@Z 1000b738     MSVCRT:dll_dllmain.obj
 0002:00001760       __sehtable$?dllmain_dispatch@@YAHQAUHINSTANCE__@@KQAX@Z 1000b760     MSVCRT:dll_dllmain.obj
 0002:00001780       __sehtable$___scrt_is_nonwritable_in_current_image 1000b780     MSVCRT:utility.obj
 0002:000017a0       .edata                     1000b7a0     j2pkcs11.exp
 0002:000017c8       rgpv                       1000b7c8     j2pkcs11.exp
 0002:000018e0       rgszName                   1000b8e0     j2pkcs11.exp
 0002:000019f8       rgwOrd                     1000b9f8     j2pkcs11.exp
 0002:00001a84       szName                     1000ba84     j2pkcs11.exp
 0002:00001a91       $N00001                    1000ba91     j2pkcs11.exp
 0002:00001a9f       $N00002                    1000ba9f     j2pkcs11.exp
 0002:00001ad7       $N00003                    1000bad7     j2pkcs11.exp
 0002:00001b0c       $N00004                    1000bb0c     j2pkcs11.exp
 0002:00001b3e       $N00005                    1000bb3e     j2pkcs11.exp
 0002:00001b71       $N00006                    1000bb71     j2pkcs11.exp
 0002:00001ba5       $N00007                    1000bba5     j2pkcs11.exp
 0002:00001be1       $N00008                    1000bbe1     j2pkcs11.exp
 0002:00001c1b       $N00009                    1000bc1b     j2pkcs11.exp
 0002:00001c57       $N00010                    1000bc57     j2pkcs11.exp
 0002:00001c8e       $N00011                    1000bc8e     j2pkcs11.exp
 0002:00001cca       $N00012                    1000bcca     j2pkcs11.exp
 0002:00001d05       $N00013                    1000bd05     j2pkcs11.exp
 0002:00001d42       $N00014                    1000bd42     j2pkcs11.exp
 0002:00001d7b       $N00015                    1000bd7b     j2pkcs11.exp
 0002:00001db8       $N00016                    1000bdb8     j2pkcs11.exp
 0002:00001df3       $N00017                    1000bdf3     j2pkcs11.exp
 0002:00001e2d       $N00018                    1000be2d     j2pkcs11.exp
 0002:00001e66       $N00019                    1000be66     j2pkcs11.exp
 0002:00001ea2       $N00020                    1000bea2     j2pkcs11.exp
 0002:00001ede       $N00021                    1000bede     j2pkcs11.exp
 0002:00001f15       $N00022                    1000bf15     j2pkcs11.exp
 0002:00001f51       $N00023                    1000bf51     j2pkcs11.exp
 0002:00001f8c       $N00024                    1000bf8c     j2pkcs11.exp
 0002:00001fc9       $N00025                    1000bfc9     j2pkcs11.exp
 0002:00002001       $N00026                    1000c001     j2pkcs11.exp
 0002:0000203c       $N00027                    1000c03c     j2pkcs11.exp
 0002:0000207c       $N00028                    1000c07c     j2pkcs11.exp
 0002:000020bb       $N00029                    1000c0bb     j2pkcs11.exp
 0002:00002102       $N00030                    1000c102     j2pkcs11.exp
 0002:00002149       $N00031                    1000c149     j2pkcs11.exp
 0002:00002184       $N00032                    1000c184     j2pkcs11.exp
 0002:000021c3       $N00033                    1000c1c3     j2pkcs11.exp
 0002:00002201       $N00034                    1000c201     j2pkcs11.exp
 0002:00002242       $N00035                    1000c242     j2pkcs11.exp
 0002:00002278       $N00036                    1000c278     j2pkcs11.exp
 0002:000022b8       $N00037                    1000c2b8     j2pkcs11.exp
 0002:000022f8       $N00038                    1000c2f8     j2pkcs11.exp
 0002:00002339       $N00039                    1000c339     j2pkcs11.exp
 0002:00002377       $N00040                    1000c377     j2pkcs11.exp
 0002:000023b2       $N00041                    1000c3b2     j2pkcs11.exp
 0002:000023ed       $N00042                    1000c3ed     j2pkcs11.exp
 0002:00002429       $N00043                    1000c429     j2pkcs11.exp
 0002:00002463       $N00044                    1000c463     j2pkcs11.exp
 0002:00002498       $N00045                    1000c498     j2pkcs11.exp
 0002:000024ce       $N00046                    1000c4ce     j2pkcs11.exp
 0002:00002509       $N00047                    1000c509     j2pkcs11.exp
 0002:00002543       $N00048                    1000c543     j2pkcs11.exp
 0002:00002584       $N00049                    1000c584     j2pkcs11.exp
 0002:000025c5       $N00050                    1000c5c5     j2pkcs11.exp
 0002:000025f9       $N00051                    1000c5f9     j2pkcs11.exp
 0002:00002632       $N00052                    1000c632     j2pkcs11.exp
 0002:0000266a       $N00053                    1000c66a     j2pkcs11.exp
 0002:000026a5       $N00054                    1000c6a5     j2pkcs11.exp
 0002:000026e4       $N00055                    1000c6e4     j2pkcs11.exp
 0002:0000271e       $N00056                    1000c71e     j2pkcs11.exp
 0002:00002757       $N00057                    1000c757     j2pkcs11.exp
 0002:0000278d       $N00058                    1000c78d     j2pkcs11.exp
 0002:000027c8       $N00059                    1000c7c8     j2pkcs11.exp
 0002:00002802       $N00060                    1000c802     j2pkcs11.exp
 0002:0000283f       $N00061                    1000c83f     j2pkcs11.exp
 0002:00002880       $N00062                    1000c880     j2pkcs11.exp
 0002:000028bc       $N00063                    1000c8bc     j2pkcs11.exp
 0002:000028f3       $N00064                    1000c8f3     j2pkcs11.exp
 0002:00002927       $N00065                    1000c927     j2pkcs11.exp
 0002:00002963       $N00066                    1000c963     j2pkcs11.exp
 0002:00002999       $N00067                    1000c999     j2pkcs11.exp
 0002:000029d4       $N00068                    1000c9d4     j2pkcs11.exp
 0002:00002a0e       $N00069                    1000ca0e     j2pkcs11.exp
 0002:00002a4b       $N00070                    1000ca4b     j2pkcs11.exp
 0002:00002d72       .idata$6                   1000cd72     kernel32:KERNEL32.dll
 0002:00002dce       .idata$6                   1000cdce     vcruntime:VCRUNTIME140.dll
 0002:00002f24       .idata$6                   1000cf24     ucrt:api-ms-win-crt-string-l1-1-0.dll
 0002:00002f46       .idata$6                   1000cf46     ucrt:api-ms-win-crt-stdio-l1-1-0.dll
 0002:00002f66       .idata$6                   1000cf66     ucrt:api-ms-win-crt-heap-l1-1-0.dll
 0002:00002f86       .idata$6                   1000cf86     ucrt:api-ms-win-crt-runtime-l1-1-0.dll
 0003:00000000       _ckpAttributesTemplate     1000d000     p11_keymgmt.obj
 0003:00000318       ?__proc_attached@@3HA      1000d318     MSVCRT:dll_dllmain.obj
 0003:00000320       _GS_ExceptionRecord        1000d320     MSVCRT:gs_report.obj
 0003:00000370       _GS_ContextRecord          1000d370     MSVCRT:gs_report.obj
 0003:00000658       ?is_initialized_as_dll@@3_NA 1000d658     MSVCRT:utility.obj
 0003:00000659       ?module_local_atexit_table_initialized@@3_NA 1000d659     MSVCRT:utility.obj
 0003:0000065c       ?module_local_atexit_table@@3U_onexit_table_t@@A 1000d65c     MSVCRT:utility.obj
 0003:00000668       ?module_local_at_quick_exit_table@@3U_onexit_table_t@@A 1000d668     MSVCRT:utility.obj
 0004:00000060       $R000000                   1000e060     j2pkcs11.dll.res
